:1000000012C02CC02BC050C6CFC528C027C026C0E8
:1000100025C024C023C022C021C020C01FC01EC0D4
:100020001DC01CC01BC011241FBECFE5D4E0DEBF25
:10003000CDBF10E0A0E6B0E0E0E3FCE102C0059037
:100040000D92AA3FB107D9F721E0AAEFB0E001C0B5
:100050001D92AC33B207E1F755DBE8CDD1CF9198D3
:100060009098899888980895899A82E08A95F1F7FE
:1000700000C00895889A82E08A95F1F700C08998B7
:1000800082E08A95F1F700C0889882E08A95F1F7BE
:1000900000C0899A82E08A95F1F700C00895889A95
:1000A000899A82E08A95F1F700C0889882E08A9563
:1000B000F1F700C0899882E08A95F1F700C00895B1
:1000C00098E0889A87FF02C0899801C0899A22E047
:1000D0002A95F1F700C0889822E02A95F1F700C030
:1000E000880F915071F7889A899882E08A95F1F784
:1000F00000C0889822E02A95F1F700C080B3869569
:10010000817081950895282F889A899832E03A95D0
:10011000F1F700C0889882E08A95F1F700C090B3AB
:1001200091FB882780F997E0889A32E03A95F1F7B9
:1001300000C0889832E03A95F1F700C0880F8199A5
:100140008160915089F7889A211102C0899A01C073
:10015000899892E09A95F1F700C0889832E03A9534
:10016000F1F700C00895CF93880F413049F4C82FAC
:10017000C60F8C2FA5DF8F3F31F491DF75DFF9CFEC
:10018000860FCF919DCFCF910895FC01680F791F05
:1001900080E048E1E617F70781F0219198E0322FDF
:1001A0003827532F517030FD84278695513009F43C
:1001B00080682695915099F7EDCF0895DC01CB0129
:1001C00081159105A105B10529F081509040A0400D
:1001D000B040D9F70895282F20779AE0299F900101
:1001E000112494E0359527959A95E1F78F70820F49
:1001F000089540E050E0E0E0FAE06F2FCFDC292FD7
:10020000042E01C0220F0A94EAF7E22B4C5F5F4FE5
:100210004031510591F78E2F0895CF93C82FC370A9
:100220006111C0614111C0681FDF80ED49DF87E0C7
:1002300047DF8C2F45DFCF9132CFEF92FF920F93A4
:100240001F93CF93DF93EC018B017A010DDF80EDDB
:1002500037DF80E035DF23DF07DF81ED31DF81E04D
:1002600052DFB9DFF70180831ADFFEDE81ED28DF80
:1002700081E049DFB0DFF801808311DFF5DE81ED39
:100280001FDF81E040DFA7DF8883DF91CF911F91DF
:100290000F91FF90EF9003CF1F93CF93DF9300D088
:1002A000CDB7DEB7182F49836A83DEDE80ED08DF25
:1002B00080E006DF4981842F9CDF02DF6A81862F80
:1002C00098DFFEDE812F95DFFBDE0F900F90DF9130
:1002D000CF911F91E4CEEF92FF920F931F93CF9394
:1002E000DF937C018B01EA01BFDE80EDE9DE84E073
:1002F000E7DED5DEB9DE81EDE3DE81E004DF6BDF32
:10030000F7018083CCDEB0DE81EDDADE81E0FBDE5A
:1003100062DFF8018083C3DEA7DE81EDD1DE81E0FC
:10032000F2DE59DF8883DF91CF911F910F91FF900B
:10033000EF90B5CE1F93CF93DF9300D0CDB7DEB74C
:10034000182F4A83698390DE80EDBADE84E0B8DE40
:10035000812F4FDFB5DE6981862F4BDFB1DE4A8109
:10036000842F47DFADDE0F900F90DF91CF911F916B
:1003700096CE1F93CF93DF931F92CDB7DEB7182F82
:1003800073DE80ED9DDE812F9BDE6EDE81ED98DEDB
:1003900080E0B9DE898383DE89810F90DF91CF9180
:1003A0001F9108951F93CF93DF931F92CDB7DEB7B0
:1003B000182F698359DE80ED83DE812F81DE69810C
:1003C000862F7EDE0F90DF91CF911F9168CE0F9325
:1003D0001F93CF93DF93DB01EC9111969C911197C2
:1003E000F0E0F92B803179F4EE7F63E0EE0FFF1F30
:1003F0006A95E1F716969C9116976CE070E0691B80
:100400007109E60FF71FF7FF07C091E0EA01988333
:10041000F195E195F10902C0EA011882883279F478
:1004200014968C91982F9076903649F086FF02C0F2
:10043000EE7F05C085FF02C0EC7F01C0E87FCF01E1
:1004400044E0969587954A95E1F7D9018C93EF7032
:10045000E801E88380E0DF91CF911F910F9108952B
:10046000CF93DF93CDB7DEB728970FB6F894DEBFF2
:100470000FBECDBF282F362F98E0E2EFF0E0DE016F
:10048000119601900D929A95E1F761E772E0469F0F
:10049000C001479F900D112468EE73E09FDB8AE056
:1004A000389F600D711D112421110CC0FE01319681
:1004B00088E08E0F9191491303C06F5F7F4F02C098
:1004C0008E13F8CFCB0128960FB6F894DEBF0FBE7F
:1004D000CDBFDF91CF910895882319F07195619573
:1004E0007109442319F03195219531096217730779
:1004F00034F081E0261737071CF080E008958FEF75
:1005000008950F931F93CF93DF93EC018B01B801F4
:100510008881DDDA88839FEF980F9D3F30F4F801E2
:100520009081983211F0903191F7DF91CF911F9126
:100530000F910895CF93DF93EC0123DABE0184EB92
:100540000EDB81E076DAC82F1CDA81E0C11101C030
:1005500080E0DF91CF9108951F93CF93DF9300D078
:10056000CDB7DEB7182F69837A830BDAD9D96981C1
:100570007A81882331F084E4F2DA113021F0D9D97C
:1005800002C082E001C080E00F900F90DF91CF9118
:100590001F9108955F926F927F928F929F92AF9278
:1005A000BF92CF92DF92EF92FF920F931F93CF9360
:1005B000DF93CDB7DEB729970FB6F894DEBF0FBE35
:1005C000CDBF5C014B013A018901DBD9B5018EEB4E
:1005D000C6DACE0101967C016C0199E0592E5E0CC1
:1005E00074DAF60181936F015E12FACF69E070E070
:1005F000C701CBDDD82E811107C09301A401B7013B
:10060000F5018081E4DE02C083E0D82E8D2D29968D
:100610000FB6F894DEBF0FBECDBFDF91CF911F9113
:100620000F91FF90EF90DF90CF90BF90AF909F9091
:100630008F907F906F905F9008956F927F928F92CE
:100640009F92AF92BF92CF92DF92EF92FF920F9361
:100650001F93CF93DF93CDB7DEB729970FB6F894EA
:10066000DEBF0FBECDBF782E5B014A01890160E07D
:1006700070E08EEB74DACE0101967C016C0199E09A
:10068000692E6E0C22DAF60181936F016E12FACF99
:1006900069E070E0C70179DDD82E811106C09401B0
:1006A000A501B701872D93DE02C083E0D82E8D2DE2
:1006B00029960FB6F894DEBF0FBECDBFDF91CF9164
:1006C0001F910F91FF90EF90DF90CF90BF90AF9070
:1006D0009F908F907F906F900895FF920F931F933C
:1006E000CF93DF93EC01F62E042F122F4AD918D99D
:1006F000882369F0BE018EE432DA8F2DD6D9802F9F
:10070000D4D98881883229F4812FCFD902C081E0E1
:1007100001C080E0DF91CF911F910F91FF9008956C
:100720000F931F93CF93DF93EC018B012AD9F8D855
:10073000882369F0BE018EEB12DAE801075F1F4FD4
:10074000C4D98993C017D107D9F780E001C081E0EF
:10075000DF91CF911F910F9108951F93CF93DF9356
:1007600000D0CDB7DEB7182F69837A830AD9D8D8DD
:1007700069817A81882371F088E4F1D9113009F018
:10078000D8D860E27EE480E090E018DD113021F0FE
:10079000E3D802C082E001C080E00F900F90DF91AB
:1007A000CF911F910895CF93DF93EC01EAD8B8D889
:1007B000882351F0BE0188EBD2D960E27EE480E06C
:1007C00090E0FCDC80E001C081E0DF91CF910895F2
:1007D000EF92FF921F93CF93DF93CDB7DEB72997A8
:1007E0000FB6F894DEBF0FBECDBF8FEF898784E2CE
:1007F000E82E81E0F82E10E08985882331F112304F
:1008000021F1BE016F5F7F4FCE0109967ADE8985A7
:100810008F3F19F08E3F39F48FEF8093770081E09E
:100820008093760012C0FE01319680E090E0219125
:10083000D701A80FB91F2C93019688309105B9F7FD
:100840001F5F88E0E80EF11CD7CF812F29960FB6E5
:10085000F894DEBF0FBECDBFDF91CF911F91FF9007
:10086000EF900895362F9091060191112CC02AE047
:10087000622F94D980930C0190930D01832F8ED910
:1008800080930E0190930F01842F88D980931001DB
:1008900090931101ECE0F1E080E090E021E04191E3
:1008A000DC01AE51BF4F3C91DC01A45EBE4F43174B
:1008B00011F02C9301C01C9201968630910579F7B6
:1008C00010920401089510921C0110921D011092C3
:1008D0001E0110921F011092200110922101089513
:1008E000CF93DF93362F2AE0622F58D980930C01E3
:1008F00090930D01832F52D980930E0190930F0195
:10090000842F4CD98093100190931101ACE0B1E099
:1009100080E090E052E063E02C91FC01EE51FF4F4B
:100920003081EC01C45EDE4F321708F45883308109
:10093000231708F4688329E048813C91423031F460
:100940004081431719F040814F5F40834881433015
:1009500031F44081431719F0408141504083408178
:10096000431308C00196119686309105A9F6DF91D0
:10097000CF9108953FE745EB71E031504040704022
:10098000E1F700C000002150B9F6ECCFCF93DF9320
:10099000EC0110920001109201011092FE001092E1
:1009A000FF0025E030E08AE09091E3009093E200C0
:1009B0009091E4009093E3009091E5009093E4001F
:1009C0009091E6009093E5009091E7009093E60007
:1009D000F901EE51FF4F80834FEF50E762E0415045
:1009E00050406040E1F700C0000021503109E1F6BD
:1009F0008AE08093E200CE0164E670E0DBD8462F07
:100A0000EAE0F0E0CE01BF01D5D8282FCB01BF012D
:100A1000D1D8922F25E030E05AE0F901EE51FF4F96
:100A20004083F901ED51FF4F8083F901EC51FF4FF5
:100A30009083F901EB51FF4F50837FEFE0E762E0D5
:100A40007150E0406040E1F700C0000021503109E2
:100A50002130310511F781E080930001809176000B
:100A6000813031F48091DF008093EB001092E2003E
:100A7000DF91CF910895109200018091E2008111E1
:100A800049C080E090E02AE03091E6003093E70032
:100A90003091E5003093E6003091E4003093E500BA
:100AA0003091E3003093E4003091E2003093E300B2
:100AB000FC01EE51FF4F20833FEF40E752E0315001
:100AC00040405040E1F700C000000196863091059B
:100AD000D9F646E151E063E271E08AE191E0ADDBF5
:100AE00080911A012AE0622F59D880930C019093CB
:100AF0000D018091230152D880930E0190930F0134
:100B0000809116014BD88093100190931101E2E17E
:100B1000F1E025C080E090E02AE03091E6003093DB
:100B2000E7003091E5003093E6003091E400309327
:100B3000E5003091E3003093E400FC01EE51FF4FFB
:100B400020833FEF40E752E0315040405040E1F712
:100B500000C00000019684309105F9F6BACF80916B
:100B6000E6008093E7008091E5008093E6008091A5
:100B7000E4008093E5008091E3008093E40080919D
:100B8000E2008093E30082918093E2008FEF90E790
:100B900022E0815090402040E1F700C0000031E0A9
:100BA000EC30F307E1F608951F920F920FB60F9203
:100BB00011242F933F938F939F93EF93FF93949AD6
:100BC00088B38E7388BB82B38F7182BB15BAE091F4
:100BD0000301F0E0E551FF4F808183BD8091040166
:100BE000893108F056C0809102018F5F823119F07F
:100BF000809302014EC0109202012091DE0080E03D
:100C000090E0FC01E45EFE4F3081313021F0309104
:100C10000401311124C0211106C0E0910401F0E06B
:100C2000EB53FF4F17C0213031F4E0910401F0E0A5
:100C3000E455FF4F0FC0223031F4E0910401F0E0A1
:100C4000ED56FF4F07C0233051F4E0910401F0E06E
:100C5000E658FF4F3081FC01E551FF4F3083309162
:100C600004013C3061F430910601311108C0FC01EF
:100C7000E45FFE4F3081FC01EE51FF4F308301965F
:100C80008630910509F0BDCF809104018F5F80937C
:100C90000401FF91EF919F918F913F912F910F90C0
:100CA0000FBE0F901F9018951F920F920FB60F92C4
:100CB00011248F939F93EF93FF93809103018630CC
:100CC00008F044C080910301E0910301F0E0EE518F
:100CD000FF4FE08195B3F0E0843030F4E559FF4FE9
:100CE0008081892B85BB18C0E05AFF4F8081892BFA
:100CF00085BB8091FD00E0910301F0E0811107C008
:100D0000E450FF4F8081882339F0AD9A05C0E6504A
:100D1000FF4F80818111AC9A80910301823081F074
:100D200030F4882359F08130D1F4C79A18C0843048
:100D300059F040F0853099F4C09A11C0C69A0FC09E
:100D4000959A0DC0969A0BC0979A09C0809103019D
:100D5000863029F48091E000813009F494988091E4
:100D600003018F5F80930301873060F010920301CD
:100D70008091FD00811104C081E08093FD0002C0DC
:100D80001092FD00FF91EF919F918F910F900FBEF8
:100D90000F901F90189580917800882309F45EC009
:100DA00080E090E021E0FC01E050FF4F2083B1990A
:100DB00003C080E090E049C0B29BFBCFB39BF9CF6A
:100DC0003FE748E351E0315040405040E1F700C078
:100DD0000000FC01E250FF4F2083B19BEACFB29BA1
:100DE000E8CFB39BE6CF3FE748E351E031504040C6
:100DF0005040E1F700C000000197D9F281E090E097
:100E0000D2CFB29B28C0B39B26C02FE738E341E086
:100E1000215030404040E1F700C00000FC01E250AA
:100E2000FF4F1082B19B17C0B29B15C0B39B13C07C
:100E30005FE728E331E0515020403040E1F700C047
:100E40000000019741F081E090E0FC01E050FF4F8D
:100E50001082B199D6CF10927800089581E090E089
:100E600021E0FC01E250FF4F2083B19903C081E0F3
:100E700090E049C0B29BFBCFB39BF9CF4FE758E35B
:100E800031E0415050403040E1F700C00000FC012B
:100E9000E050FF4F2083B19BEACFB29BE8CFB39BDA
:100EA000E6CF4FE758E331E0415050403040E1F7A2
:100EB00000C00000892BD9F280E090E0D2CFB29B35
:100EC00028C0B39B26C04FE758E321E04150504073
:100ED0002040E1F700C00000FC01E050FF4F10820D
:100EE000B19B17C0B29B15C0B39B13C03FE748E34B
:100EF00051E0315040405040E1F700C00000892BE4
:100F000041F080E090E0FC01E250FF4F1082B19987
:100F1000D6CF81E08093780008958091790088236E
:100F200019F08130C1F00895809178008823A1F0F4
:100F3000109200011092010110920201109203011F
:100F40001092FE001092FF00109200011092010119
:100F50001092780008951FCF08951F93CF93DF93C9
:100F6000EC019091DF009093EB009093EC00909354
:100F7000ED009093EE009093EF009093F00011E05D
:100F800010930001109201011092FE001092FF00D8
:100F900060E070E081E0E0DACC5DDE4F8881809334
:100FA000120125E131E047E750E066E770E045DBFC
:100FB000882329F08FEF809377001093760040917B
:100FC000150160917700809176004ADADF91CF9128
:100FD0001F91DCCC46E151E063E271E08AE191E0EF
:100FE0002CD9409116016091230180911A013ACCCD
:100FF0004BE151E064E371E082E291E06CD98091D1
:10100000DF00EBEEF0E0808381838283838384833F
:101010008583E0E0F1E010821182EEEFF0E01082D3
:10102000118240911B01609134018091220158CCC2
:101030008091E100813049F030F0823021F183303D
:1010400009F453C00895C6DF9BC080910901893718
:1010500008F4C0DF80910901893709F4C9DF809164
:101060000901833808F48EC046E151E063E271E083
:101070008AE191E0E2D840911601609123018091CC
:101080001A012EDC7DC080910901893708F4A2DFA6
:1010900080911301882371F0813071F480910901EE
:1010A000893719F480E090E058DF80910901833896
:1010B00018F0E1DC1092090180911301823009F0EF
:1010C00061C080910901893719F480E090E045DF23
:1010D00080910901833819F481E090E03EDF80912E
:1010E00009018D3808F44EC04AC080910901893742
:1010F00008F470DF80910901893709F479DF809164
:101100001301811114C080910901833880F046E1F8
:1011100051E063E271E08AE191E08FD840911601DD
:101120006091230180911A01DBDB1092090180910B
:101130001301813071F480910901833819F480E042
:1011400090E00BDF809109018D3818F094DC10924B
:101150000901809113018230A9F48091090183383B
:1011600019F480E090E0F9DE809109018D3819F4DE
:1011700081E090E0F2DE80910901873918F07BDC94
:10118000109209010895809108018823C1F080918F
:1011900006018330A0F480911A012AE0622FFED468
:1011A0008093E2009093E30080912301F7D4809331
:1011B000E4009093E5001092E6001092E700809121
:1011C00008018823D9F0809106018330B8F080911E
:1011D00022012AE0622FE2D48093E2009093E300A0
:1011E00080913401DBD48093E4009093E5008091FA
:1011F0001B01D4D48093E6009093E7008091060110
:10120000833009F477C028F4813051F08230E9F15D
:101210000895843009F4A8C0853009F4DFC008952A
:10122000B29913C080911A018F5F883118F48093AE
:101230001A0102C010921A012FEF80E792E02150AC
:1012400080409040E1F700C00000B39915C0809144
:101250001A01815080931A01B39905C0811103C00E
:1012600087E180931A012FEF80E792E021508040C0
:101270009040E1F700C00000829904C0B39B02C017
:10128000B2996CC080911A0162C0B29913C080916A
:1012900023018F5F8C3318F48093230102C01092D6
:1012A00023012FEF80E792E0215080409040E1F74A
:1012B00000C00000B39915C0809123018150809334
:1012C0002301B39905C0811103C08BE380932301EF
:1012D0002FEF80E792E0215080409040E1F700C07E
:1012E0000000829904C0B39B02C0B29971C0809182
:1012F000230167C0B29911C0809122018F5F8032B3
:1013000008F081E0809322012FEF80E792E02150E6
:1013100080409040E1F700C00000B39910C0809178
:101320002201815009F48FE1809322012FEF80E7A1
:1013300092E0215080409040E1F700C00000829987
:1013400004C0B39B02C0B29909C0809122016AE037
:1013500025D48093E2009093E30008958AE080937F
:10136000E2008093E3000895B29911C080913401A6
:101370008F5F8D3008F081E0809334012FEF80E79C
:1013800092E0215080409040E1F700C00000B39906
:1013900010C080913401815009F48CE080933401B5
:1013A0002FEF80E792E0215080409040E1F700C0AD
:1013B0000000829904C0B39B02C0B29909C0809119
:1013C00034016AE0EBD38093E4009093E500089544
:1013D0008AE08093E4008093E5000895B2990EC0FE
:1013E00080911B018F5F80931B012FEF80E792E0BC
:1013F000215080409040E1F700C00000B3990EC03A
:1014000080911B01815080931B012FEF80E792E0B8
:10141000215080409040E1F700C00000829904C054
:10142000B39B02C0B29909C080911B016AE0B6D398
:101430008093E6009093E70008958AE08093E600A9
:101440008093E7000895B29926C08091060181112A
:1014500005C0809105018F5F809305018091050192
:101460008A3079F48091E000813019F41092E00024
:1014700003C081E08093E0006091E00083E090E0B1
:10148000C8D32FEF30E782E0215030408040E1F7B1
:1014900000C000001EC0809105018823C1F080912A
:1014A00005018A30A0F48AE080930601A1DD9FEF58
:1014B00023ED30E3915020403040E1F700C00000C0
:1014C00081E080937800109206011092050110923D
:1014D0000501B3993CC080910601811105C080913E
:1014E00007018F5F80930701809107018A3029F5FA
:1014F00081E080930001809301018093FE0080933E
:10150000FF0090917900992319F01092790002C0A0
:10151000809379006091790080E090E07AD3109216
:10152000090181E0809378008FEF99E628E18150EE
:1015300090402040E1F700C000003FEF80E792E0DC
:10154000315080409040E1F700C0000034C08091ED
:101550000701882371F1809107018A3050F58AE0F4
:101560008093060180911301882319F080E090E0B8
:10157000F4DC2FEF33ED80E3215030408040E1F781
:1015800000C0000080911301823061F481E090E09E
:10159000E4DC9FEF23ED30E3915020403040E1F751
:1015A00000C0000081E08093780010920601109244
:1015B000070110920701B19963C0809108018F5F04
:1015C0008093080180910601823031F440E06091FF
:1015D000230180911A0160D680910801813049F47D
:1015E00080910601882329F0809106018F5F809306
:1015F0000601809108018A30E1F480910601811191
:1016000018C081E0809306011092E0009FEF21EE68
:1016100034E0915020403040E1F700C000001092CB
:101620000001109201011092FE001092FF008093C1
:10163000E000809106018630C8F01092E0008FEF44
:1016400090E722E0815090402040E1F700C0000088
:1016500081E08093E00040911B0160913401809112
:10166000220168D610920601109208013FEF80E730
:1016700092E0315080409040E1F700C000000895B2
:101680008091060181113BC0809108018823B9F146
:101690008091E1008F5F8093E100109209018091B9
:1016A000E100843010F01092E1008AE0809306019E
:1016B00010920001109201011092FE001092FF00A2
:1016C0008093E2008093E3001092E4009091E100A7
:1016D0009F5F9093E5008093E6008093E7002FEFF3
:1016E00034E38CE0215030408040E1F700C000003E
:1016F000109206016091E10082E090E08AD210929F
:101700000801089584B38F6384BB87B3816C87BB62
:1017100081B3806F81BB88B38E6088BB85B58360E1
:1017200085BD89B7806C89BF87B1876087B987EC31
:1017300086B995D441E061E080E06FD525E047E3CC
:1017400050E068E370E086E390E05FD141D8809399
:101750001301882321F060E070E081E0FDD62FEFD7
:1017600080E792E0215080409040E1F700C0000007
:1017700081E090E046D2813081F061E083E090E04A
:1017800048D263E082E090E044D261E081E090E002
:1017900040D261E080E090E03CD283E090E031D242
:1017A0008093E00082E090E02CD28093E10080E022
:1017B00090E027D28093790078948AE080930601A4
:1017C0008093E2008093E3001092E4009091E100A6
:1017D0009F5F9093E5008093E6008093E7002FEFF2
:1017E00083ED90E3215080409040E1F700C000007D
:1017F000109206014BE151E064E371E082E291E076
:101800006AD5D7EC17EDC1E00AE08FE3F82E90E53A
:10181000E92E22E0D22E39E6C32E46E9B42E53E05B
:10182000A52E63E9962E72ED872E809106018823FE
:1018300029F0809106018A3008F4A5DC04DE829B41
:1018400066C080910601811162C080910A018111F8
:10185000ECCF80910A018F5F80930A01809109018A
:101860008F5F80930901D6B9349BFECF16B984B13E
:1018700095B19093FB008093FA008091FA009091CB
:10188000FB008039914034F4A092DE009092DF009A
:101890008092F1008091FA009091FB008139914093
:1018A0006CF08091FA009091FB00843F914034F4F9
:1018B000D092DE00C092DF00B092F1008091FA0079
:1018C0009091FB00853F91406CF08091FA009091DF
:1018D000FB008835924034F4C093DE00F092DF00C4
:1018E000E092F1008091FA009091FB0089359240DE
:1018F00034F01092DE00C093DF000093F10098DB1B
:1019000080910901893708F090CF07DB8ECF1092C4
:101910000A018BCF8115910511F00197F1F7089518
:10192000E0913801F091390190818091370189234C
:101930000895E0913501F091360190818091370151
:10194000892B8083E0913A01F0913B019081809155
:101950003701892B80830895E0913501F09136019C
:10196000908180913701809589238083E0913A01AD
:10197000F0913B019081809137018095892380838C
:1019800008951F93CF93DF93E0913501F0913601D5
:10199000908180913701809589238083E0913A017D
:1019A000F0913B01908180913701892B808385EAFA
:1019B00095E0B0DF1FB7F894E0913A01F0913B0158
:1019C00090818091370180958923808386EC90E017
:1019D000A1DFE0913801F0913901D081C091370148
:1019E0001FBF8EED94E096DFE0913801F091390150
:1019F000808190913701982319F08D2F8C2301C09D
:101A000081E0DF91CF911F91089550933B01409366
:101A10003A017093360160933501909339018093B8
:101A2000380181E001C0880F2A95EAF780933701D9
:101A3000A8CFCF93DF93C82FDFB7F894E0913A0196
:101A4000F0913B01908180913701892B808382E066
:101A500090E060DFCC2351F0E0913A01F0913B013E
:101A600090818091370180958923808386E290E080
:101A700051DFE0913801F091390190818091370177
:101A8000892309F4C0E087E890E044DFE0913A015F
:101A9000F0913B019081809137018095892380836B
:101AA000DFBF8C2FDF91CF910895CF93DF93C82FA5
:101AB000D8E08C2F8170BDDFC6958111C068D150F0
:101AC000C1F78C2FDF91CF9108958FEFEECFDF928A
:101AD000EF92FF920F931F93CF93DF93E82E8B012A
:101AE00050DF811131C080EFE0DFD0E0C0E488EF4B
:101AF000D82EDC0E81E09DDFF82E81E09ADF88236E
:101B000019F0FF2071F022C0F1100BC0CE1530F09B
:101B1000F801808180FF05C0EC1619F0DC2FFF244E
:101B2000F3948F2D86DFF80190819695FF2011F0B8
:101B30009068F8019083C150CD11DCCF0F5F1F4F2B
:101B4000C111D5CF8D2F03C08FEF01C08EEFDF9174
:101B5000CF911F910F91FF90EF90DF900895EF923A
:101B6000FF921F93CF93DF93182FEB010ADF20978B
:101B700061F085E59ADF7E0188E0E80EF11C89912D
:101B800094DFCE15DF05D9F702C08CEC8EDF812FF4
:101B9000DF91CF911F91FF90EF9087CF991B79E054
:101BA00004C0991F961708F0961B881F7A95C9F7ED
:101BB00080950895AA1BBB1B51E107C0AA1FBB1F3C
:101BC000A617B70710F0A61BB70B881F991F5A95C9
:101BD000A9F780959095BC01CD01089597FB072E3C
:101BE00016F4009406D077FD08D0E4DF07FC05D09A
:101BF0003EF4909581959F4F0895709561957F4F24
:101C00000895E199FECF9FBB8EBBE09A99278DB3D3
:101C10000895262FE199FECF9FBB8EBB2DBB0FB63B
:101C2000F894E29AE19A0FBE01960895F894FFCFD6
:101C300002000C080D05040109030F00010203084E
:101C40000D05040C090F01FF0101939BA3ABB3BB6E
:101C5000C3CBD3DBE3EBF5EBE3DBD3CBC3BBB3AB62
:101C6000A39B9369747F8A95A2AFBAC6D2DEEAF5C8
:101C7000EADED2C6BAAFA2958A7F74693F4E5D6C28
:101C80007B8A99A8B7C6D5E4E4EAD5C6B7A8998AED
:101C90007B6C5D4E3F01152A3F54697E93A8BDD2EF
:101CA000E7F5E7D2BDA8937E69543F2A150101FAF2
:101CB00001020A0A0A0A0A0A000000FF0101FFFFE6
:0A1CC000FFFF01030406090B0C0EE0
:00000001FF
